:103800000C942A1C0C94451C0C94451C0C94451CCF
:103810000C94451C0C94451C0C94451C0C94451CA4
:103820000C94451C0C94451C0C94451C0C94451C94
:103830000C94451C0C94451C0C94451C0C94451C84
:103840000C94451C0C94451C0C94451C0C94451C74
:103850000C94451C11241FBECFE5D4E0DEBFCDBFC4
:1038600010E0A0E6B0E0ECE1FFE302C005900D92AD
:10387000A436B107D9F711E0A4E6B0E001C01D926B
:10388000A63AB107E1F70C94511F0C94001C0F925B
:10389000AF93BF93CF93DF93EF93FF93FC01EA01C4
:1038A000DB01C895099231961197D9F7FF91EF91F5
:1038B000DF91CF91BF91AF910F9008950F921F921A
:1038C0000F93AF93BF93CF93DF93EF93FF93FC01DD
:1038D000EA01DB010990199001E043D0329612977A
:1038E000C9F7FC0103E03DD005E03BD0FF91EF912B
:1038F000DF91CF91BF91AF910F911F900F900895DD
:103900000F931F93EF93FF93FC0103E02AD000E88D
:1039100010E0E00FF11FE617F707B9F7FF91EF91FD
:103920001F910F9108950F930F9222D0082E09E056
:1039300018D00F900F9108950F930F92EF93FF936C
:1039400017D0FC0160935700C895802DFF91EF912F
:103950000F900F9108950F930BD001E102D00F91BA
:103960000895E199FECF00935700E895FFFF00000E
:103970000091570000FDFCCF089583E089B98AB11A
:1039800088618AB908958AB1877E8AB908958CB909
:103990005E9BFECF5E9A08958CB1992708958BB1F6
:1039A0009927807890700895EF92FF920F931F935C
:1039B000CF93DF937B01C0E0D0E0C617D70770F448
:1039C0008C010E94CF1C8823E1F30E94CC1CF801DB
:1039D00081938F012196CE15DF0598F381E090E069
:1039E000DF91CF911F910F91FF90EF900895EF928B
:1039F000FF920F931F93CF93DF937C018B01C0E065
:103A0000D0E0C017D10738F4F70181917F010E94FF
:103A1000C71C2196F6CF81E090E0DF91CF911F91F6
:103A20000F91FF90EF900895EF92FF920F931F93E5
:103A3000CF93DF937C0100E010E00817190788F4AA
:103A4000C0E0D0E000000E94CF1C882351F42196F2
:103A500083E0CB36D807B0F30F5F1F4F0E151F055D
:103A600078F3DF91CF911F910F91FF90EF90089520
:103A70000E94C31C0E9400000895DF92EF92FF9203
:103A80000F931F93CF93DF93CDB7DEB72197DEBFA0
:103A9000CDBF8C017B011982D98061E070E0CE013D
:103AA000860F971F0E94D41C89818B31B1F761E08A
:103AB00070E0C8010E94D41C61E070E0CE01860F66
:103AC000971F0E94D41C89819927182F002761E035
:103AD00070E0CE01860F971F0E94D41C8981080FC9
:103AE000111D61E070E0CE01860F971F0E94D41C6B
:103AF00089818E30B9F4C8010196BC01C7010E94CA
:103B0000D41C98018FEF0F3F180779F0F7018191CE
:103B10007F01D82621503040FFEF2F3F3F07B1F7FC
:103B2000DD2019F080E090E001C0C8012196DEBFE1
:103B3000CDBFDF91CF911F910F91FF90EF90DF905C
:103B40000895CF92DF92FF920F931F93CF93DF934D
:103B5000182FEB016A018BE10E94C71C4BE1F42E88
:103B6000812F0E94C71CF1260D2F1127802F0E9444
:103B7000C71CF0268C2F0E94C71CFC268EE00E94DA
:103B8000C71C8EE0F82621978FEFCF3FD80759F05A
:103B9000F60181916F01F8260E94C71C2197FFEF63
:103BA000CF3FDF07A9F78F2D0E94C71CDF91CF9170
:103BB0001F910F91FF90DF90CF9008959927813941
:103BC000910559F08239910524F48039910529F045
:103BD00008C08239910519F004C082E003C087E073
:103BE00001C080EC99270895BF92CF92DF92EF92A7
:103BF000FF920F931F93CF93DF93B82E8B01FB019E
:103C00008081C82FDD27C231D10509F46DC0C331D1
:103C1000D105DCF4C330D10509F44DC0C430D10561
:103C200044F4C130D10579F1C230D10509F44AC05C
:103C300004C1C630D10509F44AC0C630D1050CF420
:103C4000FCC060970CF4F9C055C0C531D10509F42A
:103C5000C8C0C631D10544F4C331D10509F472C0DE
:103C6000649709F44AC0E9C0CA31D10509F4D7C044
:103C7000CB31D10524F4669709F49AC0DEC06B9766
:103C800009F4C4C0DAC0FB01118288E0828381E4B8
:103C9000838386E5848382E5858389E4868383E55F
:103CA000878380E580878FE5818782E38287AB0108
:103CB0006BE070E0C8C0FB0181810E94DE1DF8014D
:103CC000828301C0FB011182A801BE01BCC0FB01BF
:103CD00083819927982F88272481820F911D9093A3
:103CE000A5018093A40107C060E070E480E090E04B
:103CF0000E94801CF8011182A3C0FB0181819927D9
:103D0000D82FCC2782819927C82BD92B1182CB01A0
:103D100002962091A4013091A501AC01BE01C90118
:103D2000880F991F0E94471CF801EC0FFD1F12829B
:103D30009E01369527958091A4019091A501820F4F
:103D4000931F49C0FB0181819927D82FCC278281FD
:103D50009927C82BD92BCC24DD24CC16DD06D8F42A
:103D6000FAE0EF2EF12CE60EF71E8091A40190915F
:103D7000A501880F991FA70160E870E08C0D9D1DBB
:103D80000E945E1C80E890E0C80ED91EE80EF91E65
:103D9000CC16DD0650F30E94AB1CF8011182D695BB
:103DA000C7958091A4019091A5018C0F9D1F29C0FA
:103DB000FB0181819927D82FCC2782819927C82B95
:103DC000D92B1182EC0FFD1F12828091A4019091DA
:103DD000A5018C0F9D1F9093A5018093A4012396AC
:103DE00073CFFB0181819927382F22278281992760
:103DF000282B392B11828091A4019091A501820F6B
:103E0000931F9093A5018093A4011AC0FB01118216
:103E10008481E82FFF27E05AFF4F808107C0FB0114
:103E2000118269E081E090E00E949C1CF80182838D
:103E30001382A80164E070E006C089ECF801818378
:103E4000A80162E070E08B2D0E94A11DDF91CF914F
:103E50001F910F91FF90EF90DF90CF90BF9008954A
:103E6000CF93DF93CDB7DEB72197DEBFCDBF69E03B
:103E700081E090E00E949C1C992784FF09C08F7EFE
:103E80000E94931C05C064E670E089810E94F41DC5
:103E900064E670E0CE0101960E943D1D892B99F3E6
:103EA000F7CFCFE5D4E0DEBFCDBFCEE1F894AEEFE3
:103EB000B1E00E94851F802D843B71F4AFEFB1E02B
:103EC0000E94851F802D833C39F4ADEFB1E00E9444
:103ED000851F802D992781BF0E94BD1C0E94CC1C8C
:103EE00084E690E00E94141D0E94CF1C882319F0E4
:103EF0000E94301F04C0C150C8BBCC2389F70E9468
:103F0000381D80E090E00C948D1FE199FECFBFBB7F
:0C3F1000AEBBE09A11960DB20895FFCFF1
:043F1C001E940300EC
:0400000300003800C1
:00000001FF
